:100000000C9496010C94BE010C94BE010C94BE019C
:100010000C94BE010C94BE010C94BE010C94BE0164
:100020000C94BE010C9437030C940C230C94BE2149
:100030000C94BE010C94BE010C94BE010C94BE0144
:100040000C94470A0C94BE010C94BE010C94BE01A2
:100050000C94BE010C94BE010C94BE010C94DA19F0
:100060000C94BE010C94B31E0C94F61E0C94BE01AD
:100070000C94BE010C94BE010C94BE010C94BE0104
:100080000C94BE010C94BE010C94BE010C94BE01F4
:100090000C94BE010C94BE010C94BE010C94BE01E4
:1000A0000C94BE010C94BE010C94BE017D1283120F
:1000B000891290129E12C012DE12E31AE61AD91AA1
:1000C000DD1A071B071B071BEA1AEE1AF21AF81AA9
:1000D000FC1A071B021B434C49206E6F742061768B
:1000E00061696C61626C652C2075736520636F6E4D
:1000F000666967757261746F72210000000002000A
:10010000080E0000030401000B00000000000000C6
:100110000000000000000000000408020110408000
:1001200040102040804080080204018040201002DE
:10013000011080102040400404040404030405025C
:100140000202020403020202020606060606060472
:100150000402020204000000002300260029002CF3
:10016000002F0000000000250028002B002E003189
:100170000000000000240027002A002D00300008A5
:100180000B0002020201000904000001020200004B
:1001900005240010010524010101042402060524A0
:1001A0000600010705810310004009040100020A4E
:1001B000000000070502024000000705830240001E
:1001C0000000C18081C112010002020000404123F1
:1001D000368000010102000112010002000000400F
:1001E0004123368000010102000118034100720022
:1001F0006400750069006E006F0020004C004C0028
:1002000043002203410072006400750069006E0023
:100210006F0020004C0065006F006E0061007200EE
:1002200064006F00040309040000000000000000E7
:100230002A2B280000000000000000000000000041
:1002400000000000000000002C9EB4A0A1A2A43475
:10025000A6A7A5AE362D3738271E1F20212223241E
:100260002526B333B62EB7B89F8485868788898ABA
:100270008B8C8D8E8F909192939495969798999A56
:100280009B9C9D2F3130A3AD350405060708090A54
:100290000B0C0D0E0F101112131415161718191A36
:1002A0001B1C1DAFB1B0B500090402000103000022
:1002B00000092101010001226500070584034000B7
:1002C0000105010902A1010901A100850105091922
:1002D000012903150025019503750181029501751A
:1002E00005810305010930093109381581257F751C
:1002F0000895038106C0C005010906A10185020514
:100300000719E029E7150025017501950881029577
:1003100001750881039506750815002565050719FF
:100320000029658100C0941CE41FA82411241FBE6D
:10033000CFEFDAE0DEBFCDBF12E0A0E0B1E0ECEF3E
:10034000FBE402C005900D92AA35B107D9F715E07C
:10035000AAE5B2E001C01D92A831B107E1F713E0B0
:10036000CCE2D3E004C02297FE010E947125C63280
:10037000D107C9F70E9420200C94FC250C940000A2
:1003800080910008909101088737974709F0A89558
:100390000895DC01ED91FC910190F081E02D09952B
:1003A000089520919C0330919D03382748E0C901AE
:1003B000880F991F37FF06C09C0151E2252750E1A5
:1003C000352701C09C01415091F730939D03209344
:1003D0009C03089588E380939E0380E092ECA1E063
:1003E000B0E080939F039093A003A093A103B093E8
:1003F000A20387E08093AB0380EC92E9ADEEB9E114
:100400008093A3039093A403A093A503B093A603A2
:1004100085E08093AC038DEE9EEFADEABEED809358
:10042000A7039093A803A093A903B093AA03EDEAAE
:10043000F3E080E090E0863028F4DC01AC5DBD4F55
:100440002C9101C020E0219301968831910599F704
:1004500082E08093C5038AE08093C603089580EC10
:1004600091EDA8E9BBE18093E3039093E403A093AB
:10047000E503B093E60380E090E0A0E0B0E5809370
:10048000E7039093E803A093E903B093EA03EBEE4C
:10049000F3E080E081938F5F8031E1F70895A0E081
:1004A000B0E0E5E5F2E00C943A25D82F0E94301A2E
:1004B0006115710581059105C9F30E94DD25109232
:1004C000A7031092A8031092A9031092AA03C4E0F4
:1004D000812C912C54018A94C090A703D090A8033A
:1004E000E090A903F090AA03FE2CED2CDC2CCC2488
:1004F0000E94D825A50194010E9419256C0D7D1D2F
:100500008E1D9F1D6093A7037093A8038093A9037A
:100510009093AA03C15001F7DD2309F450C00DEAFE
:1005200013E0E801A12CB12C62E3C62ED12CE12C02
:10053000F12C8881882309F442C0B39419F40E94F5
:10054000EA013DC00E94D825A70196010E94192505
:10055000E1E0E60FADEAB3E08A2F801B8A1520F4B4
:100560008D918E13F9CFE9CF2091AC0330E0A0E15B
:10057000B7E20E94B1249B01AC01AE2FB0E00E9413
:10058000C0244090A3035090A4036090A5037090F2
:10059000A603640D751D861D971D4090E3035090C2
:1005A000E4036090E5037090E6034616570668067C
:1005B000790618F2E993A39488E1A812BACFCDB7CF
:1005C000DEB7E0E10C94562580919B03813019F44D
:1005D00082E080939B0380919B03833019F484E035
:1005E00080939B03089588E08093C10061E08AE0D6
:1005F0000E94081B60E08AE00E94411B089500975A
:10060000C9F09C0140E050E068E478EE81E090E0C1
:100610000E9419252F3F31054105510529F020F091
:100620002FEF30E040E050E02093D1008091C000F7
:10063000806103C08091C0008F7E8093C0000895C8
:10064000219A229A239860E08BE00E94081B61E0C7
:100650008CE00E94081B0895EBE6F0E08081806842
:100660008083E8E6F0E080818160808308951F92B6
:100670000F920FB60F9211242F933F934F935F93D6
:100680006F937F938F939F93AF93BF93EF93FF935A
:100690001F9B0E94E402FF91EF91BF91AF919F9148
:1006A0008F917F916F915F914F913F912F910F901B
:1006B0000FBE0F901F901895A1E0B0E0E2E6F3E0C6
:1006C0000C9447251FB791E090939A03F89489837F
:1006D0000E94C00198E1909360008981809360003E
:1006E00081110E94C0011FBF2196E3E00C94632595
:1006F0008F929F92AF92BF92CF92DF92EF92FF9232
:10070000CF93FC01C0A5EC2FE770F0E0E45EFD4F55
:10071000A081B0E0C7FF03C024E130E002C02FE0B9
:1007200030E0FC0197A183E1989FF0011124E25C85
:10073000FE4F80809180A280B380A20FB31F20E47F
:100740003FE14DE750E00E94CB24A50194010E94B7
:10075000F7248C2F887149F469017A01E0EDCE0EFF
:10076000E7E0DE1EE11CF11C1BC0C7FF05C060E412
:100770007AE88CE29EE004C060E07EEE8AEB9BE0CB
:1007800069017A01F8EBCF0EFBE0DF1EE11CF11CE2
:10079000A50194010E94F724C20ED31EE41EF51E8B
:1007A000C701B60169517C4F8F4F9F4F28EE33E050
:1007B00040E050E00E94F724A8EEB3E00E94C0247D
:1007C000CF91FF90EF90DF90CF90BF90AF909F9030
:1007D0008F9008958F3F910551F048F0811522E0E8
:1007E000920738F08115934030F482E0089580E05C
:1007F000089581E0089583E00895A0E0B0E0E3E08B
:10080000F4E00C944325EB018A01B82FB695A0E0E3
:1008100028813981F80120832A813B8121832C8121
:100820003D8122832E813F812383688179814A81A2
:100830005B812C813D81EE81FF819F2F9295990FE5
:10084000990F907C272F2370922B252F2370220F36
:10085000220F922B232F23702295207F922BF801B9
:1008600094830B5F1F4F2896AF5FBA1788F680FFFF
:1008700024C0888199810E94EA03D82E8A819B81B5
:100880000E94EA03E82E8C819D810E94EA03F82EE3
:100890008E819F810E94EA03F0E4DF9EA001112473
:1008A00090E1E99E90011124242B282BE4E0FE9E88
:1008B000B0011124262BF8012083CDB7DEB7E7E085
:1008C0000C945F25803223E0920708F1883E23E0F4
:1008D000920740F48F519340E4E096958795EA950E
:1008E000E1F70895803D27E0920718F48C5D93406E
:1008F0000895883928E0920768F4885C974074E08E
:10090000969587957A95E1F78D509C4F089580E0F4
:1009100090E008958FEF93E008958C30910540F4B6
:10092000A4E0880F991FAA95E1F7885D9C4F089570
:10093000843F23E0920718F484529C4F0895811558
:1009400024E0920740F48657934FF4E0880F991FF4
:10095000FA95E1F7089580E998E008959C013695AD
:10096000279525753575821B930B9C012373337373
:10097000969587959695879583739373820F931FAA
:100980009C0154E0369527955A95E1F7280F391FB9
:100990002F703F7041E051E0249FC001259F900DD2
:1009A000349F900D1124892F08952998882319F0D8
:1009B00000002A9A02C000002A980000299A00002C
:1009C0000895299A000083B12998000083FB8827A5
:1009D00080F90895CF93DF93D82F5E9A29985E9877
:1009E000C8E08D2F80780E94D504DD0FC150C9F773
:1009F0002998DF91CF9108958F770E94EA04089596
:100A0000CF93DF93D82FC8E08D2F80780E94D50434
:100A1000DD0FC150C9F72998DF91CF910895CF9389
:100A2000DF932998C8E080E0D82FDD0F0E94E10411
:100A30008D0FC150C9F7DF91CF9108950E94FC043A
:100A40000E940F055E9A0895A1E0B0E0EAE2F5E0A9
:100A50000C944825806869830E94EA046981862F86
:100A60000E9400055E9A2196E2E00C946425CF93E3
:100A7000C091A703C827E82FF0E0E256FC4F678536
:100A800089E70E9424056C2F8DE30E9424056C2FBA
:100A900082E40E942405CF91089586E20E941E05FB
:100AA0000895CF93DF93EC016C818CE10E942405C3
:100AB0006D818DE10E9424056E818EE10E942405E6
:100AC0006F8180E20E942405688581E20E942405EE
:100AD000698582E20E9424056A8583E20E942405DA
:100AE0006B8584E20E9424056C8585E20E942405C2
:100AF0006D858AE20E9424056E858EE60E9424059B
:100B00006F858FE60E942405688980E70E9424058E
:100B1000698981E70E9424056A8982E70E94240589
:100B2000DF91CF910895CF92DF92EF92FF92CF9312
:100B3000DF936B017C01C11488E3D8068CE9E806D9
:100B40008CE1F80628F5C701B60120E836E948E946
:100B500050E00E94F724E901689760E879E687E6AB
:100B60009FEF0E94D3246C0D7D1D8E1D9F1DF2E012
:100B7000660F771F881F991FFA95D1F721E732E09A
:100B800040E050E00E94F724F22EE32E80E421C0E2
:100B9000C701B60120E03DE241E351E00E94F724A5
:100BA000E901689760E073ED8EEC9EEF0E94D3241C
:100BB0006C0D7D1D8E1D9F1D660F771F881F991F51
:100BC00021E732E040E050E00E94F724F22EE32ECD
:100BD00080E66C2F6F71680F85E70E9424056E2DEB
:100BE00086E70E9424056F2D87E70E942405DF9188
:100BF000CF91FF90EF90DF90CF900895682F8DE612
:100C00000E94240508958F929F92AF92BF92CF9237
:100C1000DF92EF92FF92CF93DF93D82F83E00E9471
:100C20001E058093990384E00E941E05809398031B
:100C300060E086E00E94240561E087E00E942405D0
:100C40006FE789E00E94240565E08AE00E942405A0
:100C500065E18BE00E94240562E18CE00E9424059E
:100C60006DEF8DE00E94240560E08EE00E94240577
:100C7000DD2319F08BE291E008C02091C50333E138
:100C8000239FC0011124825C9E4F0E9451056CE895
:100C900080E30E9424056FE082E30E94240562E461
:100CA00083E30E9424058091C60387FF02C064E1AC
:100CB00001C06AE084E30E9424056AE285E30E94A1
:100CC00024056DE286E30E94240564ED87E30E941B
:100CD000240560E088E30E94240560E089E30E9427
:100CE0002405D11109C0C090A703D090A803E090BB
:100CF000A903F090AA0307C0C5E9CC2EC1ECDC2EF5
:100D0000ED2CCEEDFC2ECAE38F2C9924AA24BB2413
:100D1000682D8C2F0E942405682D85E08C0F0E9481
:100D20002405FE2CED2CDC2CCC24CF5FCE3361F7D8
:100D30006FEF83E40E9424056FEF84E40E94240592
:100D40006FEF85E40E9424056FEF86E40E9424057E
:100D5000DD2311F066E002C06091AB038DE60E94D6
:100D6000240560E089E70E9424056091AC038AE7CE
:100D70000E94240560E083E70E94240560E084E788
:100D80000E942405D11109C06091A3037091A403AE
:100D90008091A5039091A60304C060EC72E98DEEEA
:100DA00099E10E949305DF91CF91FF90EF90DF9042
:100DB000CF90BF90AF909F908F90089561E087E0B3
:100DC0000E94240564E28EE70E94240563E088E027
:100DD0000E94240560E088E00E94240565E087E029
:100DE0000E94240562E085E00E94240583E00E94C1
:100DF0001E058093990384E00E941E05809398034A
:100E0000089583E00E941E058093990384E00E9468
:100E10001E058093980361E087E00E9424056AE044
:100E200070E080E090E00E94531A0E94DE0600000D
:100E30000895CF92DF92FF920F931F93CF93DF938A
:100E40001F92CDB7DEB7082F162F8EE399830E942D
:100E50002405F02EC02E9981D92E8C2D8F19811743
:100E600038F4F60161916F018FE70E942405F5CFF8
:100E700064E085E00E94240583E00E941E058093C3
:100E8000990384E00E941E05809398030E94301A03
:100E900060939403709395038093960390939703C4
:100EA00069E087E00E94240581E080939B030F9016
:100EB000DF91CF911F910F91FF90DF90CF90089518
:100EC0000F931F930E94190780919B03813099F41F
:100ED0000E94301A0091940310919503209196037B
:100EE00030919703601B710B820B930B603A76482D
:100EF0008140910548F380919B03813031F467EA8A
:100F000071E086E094E00E94381D1F910F910895D2
:100F10000F931F9380919B03823021F410929B03C7
:100F200081E020C080919B038130D9F40E94301A67
:100F300000919403109195032091960330919703AB
:100F4000601B710B820B930B613A764881409105CF
:100F500040F061E087E00E94240510929B0382E04C
:100F600001C080E01F910F910895CF93DF93EC01B2
:100F70004AE050E06D2F70E086E094E00E94FD1D95
:100F80006EE286E094E00E940A1DBE0184E0769540
:100F900067958A95E1F76F7077274AE050E086E021
:100FA00094E00E94FD1DDF91CF910895D82FC0E0FD
:100FB000CD1780F45F9A64E670E080E090E00E94D4
:100FC000531A5F9864E670E080E090E00E94531A44
:100FD000CF5FEECF6CE271E080E090E00E94531AA8
:100FE000E6CF0F931F93CF93DF93EC01062F15E00D
:100FF000115051F0CE010E94E625081741F0602FF4
:10100000CE010E94EE25F4CF82E00E94D607DF9148
:10101000CF911F910F910895A0E0B0E0E2E1F8E0D8
:101020000C943A25482E562EC0E0D0E0612C712C4D
:10103000E12CF12C00E010E041100CC06090FC03AA
:1010400086E4689E3001112459E1E52EF12C02EE70
:1010500013E01EC091E049120FC06090FC03E6E46B
:101060006E9E30011124FBE16F0E711C49E2E42EEB
:10107000F12C0EE913E00CC082E0481209C028E10F
:10108000622E77247394EE24E394F12C0BEF13E09B
:1010900043018C0E9D1E10929D0310929C033401FF
:1010A000A62CA818B12CC30101966C01AE14BF0484
:1010B000A8F4A00EB11E511006C0C3010E94E6257F
:1010C000F501808305C0F5016081C3010E94F1072D
:1010D000F50180810E94D1013601E2CFC301511098
:1010E00018C0C3010E94E625B82EC6010E94E6255D
:1010F0002B2D30E0322F2227282B80919C039091BA
:101100009D038217930779F4C0E0D0E055245394EF
:1011100093CF360160919D030E94F10760919C037B
:10112000C6010E94F107C05EDE4FC13E92E0D907C2
:1011300008F482CF852DCDB7DEB7E0E10C945625BB
:1011400061E082E00E940C08089560E082E00E9465
:101150000C088091FB03853028F084E08093FB032A
:101160000E94A0088091FB038093FC03089561E036
:1011700080E00E940C0861E081E00E940C08089564
:1011800060E080E00E940C08882351F060E081E07C
:101190000E940C08882321F080919E03883349F037
:1011A0000E942F020E94EA0181E00E944F020E94E9
:1011B000B7080895CF93C82F0E94301A6093580340
:1011C0007093590380935A0390935B03C0936D030C
:1011D000CC2329F040E051EE60E070E004C040E82C
:1011E00055E260E070E088E594E00E94631FCF91D3
:1011F000089590915C03492F4F7050E0BA016F5FE2
:101200007F4F292F30E0E4E035952795EA95E1F707
:101210006217730759F0FA01E35AFC4F808381E0AB
:10122000890F8F70907F892B80935C0308956EE700
:1012300070E088E594E00E94C9010895A3E1B1E05F
:10124000E4E2F9E00C943B25EDEAF3E0712C8191A6
:10125000882321F0739428E17212F9CF63EB71E0D7
:1012600086E094E00E94381D4AE050E0672D86E059
:1012700094E00E94041E80E00E9403060E94DE06A5
:101280008E010E5F1F4FC12CD12C7601C3946624B2
:101290006A945C2C0E94241A4B015C012091AC03DF
:1012A00030E0A0E1B7E20E94B1249B01AC01C7018C
:1012B000B6010E94D3242091A3033091A40340914E
:1012C000A5035091A603620F731F841F951F2091E1
:1012D000E3033091E4034091E5035091E6032617C0
:1012E00037074807590718F4F801608225C08C2D8C
:1012F0000E94370561E070E080E090E00E94531AA0
:10130000F80110820E94241A681979098A099B0938
:10131000643F71408105910540F40E944D05F8013C
:101320009081981778F78083EDCF50FE03C04698E0
:101330005F9A02C0469A5F982FEFC21AD20AE20A59
:10134000F20A0F5F1F4F8FEFC816D104E104F104BA
:1013500009F09FCFCE019395FC01D82E7FEF68EC6A
:101360002E2F281B271510F051E056C0DE011296D3
:1013700051E02FEF41E03D91321710F0322F01C0C4
:10138000452F5F5F5F3F11F0232FF5CF4193242F4F
:1013900030E0A1E0B0E0AC0FBD1FA20FB31F5C9323
:1013A000413079F0DE01A20FB31F5C93423049F067
:1013B000AFEFBFEFAC0FBD1FA20FB31F6C934E3F3B
:1013C00078F6A2E0B0E0AC0FBD1FA20FB31F7C9374
:1013D0004D3F30F6A3E0B0E0AC0FBD1FA20FB31F2E
:1013E0006C93BECF452F242F30E0FC01E20FF31F9A
:1013F0006081AFEFB0E0AC0FBD1FA20FB31F2C9107
:10140000621748F44150DC01A40FB11D2C912083D8
:101410006C934111E8CF5F5F571520F3372D369558
:1014200020E0231770F4DC01A20FB11D4C91522F64
:10143000530FFC01E50FF11D50815C9340832E5F3B
:10144000F0CFFDEAEF2EF3E0FF2E8C01802F8D19F7
:10145000871598F4F801C1908F014AE050E06C2D97
:1014600086E094E00E94F51D6CE286E094E00E9424
:101470000A1DF701C1927F01E9CF86E094E00E9446
:10148000121D81E0CD5EDE4FEFE00C9457251F92D8
:101490000F920FB60F9211241F932F933F934F93E8
:1014A0005F936F937F938F939F93AF93BF93CF93EC
:1014B000DF93EF93FF93C0918600D09187008091D6
:1014C00017039091180320913903211155C09E01F3
:1014D000281B390B8091E7039091E803A091E90361
:1014E000B091EA0385FD02C036952795253C49E079
:1014F0003407B8F140910A0150E060E070E02CE15F
:10150000B695A795979587952A95D1F70097A10548
:10151000B10521F481E090E0A0E0B0E084179507E8
:10152000A607B707D8F480910A018F3FB9F040E0D1
:1015300080910A01481780F4842F90E0880F991F4A
:10154000FC01E75EFC4F20813181FC01E55FFE4F2D
:10155000318320834F5FECCF10923A0310920A013F
:101560000BC02D3B82E0380720F080910A018031CA
:10157000D8F08FEF80930A01D0931803C09317031C
:10158000FF91EF91DF91CF91BF91AF919F918F919B
:101590007F916F915F914F913F912F911F910F908C
:1015A0000FBE0F901F90189510910A0181E0810FD6
:1015B00080930A01C9010E946204E12FF0E0EE0F5E
:1015C000FF1FE75EFC4F91838083D6CF83E080933B
:1015D00080008AE9809381008091E70386FD05C041
:1015E000809181008064809381008FEF9FEF9093C2
:1015F00089008093880080916F00806280936F00E3
:1016000008950E94A5088091FC03843011F4109283
:10161000FC0308956F3018F086958058089589E08E
:10162000689F802D11240895A0E0B0E0EAE1FBE07E
:101630000C944225C82F0E94301A0091C8021091C4
:10164000C9022091CA023091CB026B017C01C01A01
:10165000D10AE20AF30A9701860149E8C41643E178
:10166000D406E104F10410F01092CC026093C80299
:101670007093C9028093CA029093CB0220913903E0
:101680008FEF820F8230D8F5E091CC02EE2309F47F
:101690004EC1E13011F482E0B8C1E03108F034C14C
:1016A00081E08E0F8093CC02F0E0E75EFC4FC083B8
:1016B000803109F0ACC1EBE1F3E0213029F4A181E4
:1016C000A695A695808108C080819181A92FA695B5
:1016D000A695A69596958795A03148F4B0E090E040
:1016E000AA0FBB1FA55FBE4F11969C938E931092BD
:1016F0003A03329683E0E932F807F9F688C12330DD
:1017000009F005C1E091CC02E11104C0CF3009F02D
:101710007EC10DC1E83148F481E08E0F8093CC0288
:10172000F0E0E85EFC4FC08372C1E83109F0ECC024
:10173000C111EAC040E050E0ABE0CA01B3E0880F5D
:10174000991FBA95E1F7A49F9001A59F300D112430
:10175000F901E75EFC4F6081E1817E2F777075951E
:101760006795FC01EE0FFF1FE55FFE4F71836083FD
:10177000F901E65EFC4FB081B695B695B695E1816C
:10178000FE2FF295FF0FF07E6F2F6B2BE695E695FF
:10179000E6957E2F777075956795FC01EE0FFF1F1C
:1017A000E35FFE4F71836083F901E55EFC4FB0811A
:1017B000B295B695B695B370C181DC2FDD0FDD0F04
:1017C0006D2F6B2BC295C695C695C370E281E170F3
:1017D000EE0FEE0F7E2F7C2B75956795FC01EE0FBB
:1017E000FF1FE15FFE4F71836083F901E35EFC4FF1
:1017F000B081B695E181FE2FF795FF27F7956F2F02
:101800006B2BE6957E2F777075956795FC01EE0F33
:10181000FF1FEF5EFE4F71836083F901E25EFC4FB4
:10182000B081B295BF70E181FE2FF295F07F6F2FEE
:101830006B2BE295EF707E2F777075956795FC01A5
:10184000EE0FFF1FED5EFE4F71836083F901E15ED5
:10185000FC4FB081BB1FBB27BB1FC181DC2FDD0F3D
:101860006D2F6B2BCC1FCC27CC1FE281E370EE0FCA
:101870007E2F7C2B75956795FC01EE0FFF1FEB5EAD
:10188000FE4F71836083F901EF5DFC4FB081B69527
:10189000B695E181FE2FF295FF0FFF0FF07C6F2FC1
:1018A0006B2BE695E6957E2F777075956795FC0115
:1018B000EE0FFF1FE95EFE4F71836083F901EE5D5D
:1018C000FC4F20812295269527703181E32FEE0F62
:1018D000EE0FEE0F6E2F622B732F72957695777049
:1018E00075956795FC01EE0FFF1FE75EFE4F718354
:1018F00060834F5F5F4F4230510509F01ECF8091EA
:101900002F0383FF10923A031092CC0280C0243040
:1019100009F07DC06091CC0261110BC0C83AB1F4EE
:1019200010929D0310929C0388EA0E94D10181E0ED
:101930006CC0613019F4C093C70204C0623031F446
:10194000C093C6028C2F0E94D1015AC0E091C602FA
:101950002E2F30E0220F331F462F50E0C901029690
:10196000841795073CF0633268F7FA01EA5EFC4F92
:10197000C083E8CF2D5F3F4F8C2F90E060919C0398
:1019800070919D034217530749F4982F88278627A3
:10199000972790939D0380939C0332C06817790723
:1019A00069F58091C702813049F5E13118F080E195
:1019B0008093C602F090C602CAE1D3E000E010E0D6
:1019C0000F15D0F4FE013197808190E0982F882781
:1019D0002881822B63E0969587956A95E1F70E94AE
:1019E0006204F801EE0FFF1FE55FFE4F91838083D5
:1019F0000F5F1F4F2296E4CF10923A031092CC0251
:101A00008091CC02882319F08F5F8093CC02CDB7F0
:101A1000DEB7E8E00C945E25E82FF0E0EE51FC4FD5
:101A2000E185E03150F4F894F0E0EE0FFF1FE55F40
:101A3000FE4F8081918178940895E03121F0E13169
:101A400069F483E001C082E00E94741B892B19F0C5
:101A500084EF93E008958CE090E0089580E092E0B8
:101A60000895A2E2B0E0E7E3FDE00C9438259E0182
:101A70002F5F3F4F80E1D9011D928A95E9F761EE12
:101A800071E086E094E029A33AA30E94381D0E94E9
:101A900001071D8A1E8A1F8A188E312C212C00E016
:101AA000812C912C540170E4472E71EE572E7DE964
:101AB000672E78E1772EE0E5CE2EE3ECDE2EE12CEA
:101AC000F12C84EF91E0A0E0B0E08D8F9E8FAF8F7E
:101AD000B8A380EC91EDA8E9BBE1898F9A8FAB8F19
:101AE000BC8F80E491EEADE9B8E1898B9A8BAB8B2A
:101AF000BC8B86E094E00E949D1B892B09F4E1C019
:101B000086E094E00E94C11B9C0133272C323105F2
:101B100009F442C0ACF42332310509F0ABC019829C
:101B20001A821B821C821D821E821F8218861986C1
:101B30001A861B861C861D861E861F86188A60C014
:101B40002434310529F02335310509F4B2C092C09F
:101B500064E486E094E00E940A1D2AE030E040E45C
:101B600051EE6DE978E186E094E00E94981D6CE208
:101B700086E094E00E940A1D2AE030E040EC51ED3E
:101B800068E97BE186E094E00E94981D6CE286E0C3
:101B900094E00E944A1DADCF0F5F043009F0A9CF39
:101BA00029813A814B815C81A8EEB3E00E94C02478
:101BB000698B7A8B8B8B9C8B2D813E814F815885D5
:101BC0000E94C024698F7A8F8B8F9C8F29853A85DC
:101BD0004B855C852D8F3E8F4F8F58A32D853E857D
:101BE0004F8558890E94C0246B017C0160323EE41D
:101BF00073078105910530F462E38CE10E942405AE
:101C000000E077CF603345E774078105910510F454
:101C100062E2F3CF60345CE975078105910510F449
:101C200066E2EBCF80E5C81683ECD806E104F10448
:101C300010F462E1E2CF90E6C9169AEED906E1040B
:101C4000F10410F465E1D9CFA0E7CA16A1E1DA06E4
:101C5000A1E0EA06F10410F461E0CFCFB0EACB16C0
:101C6000B6E8DB06B1E0EB06F10410F463E0C5CFA3
:101C700065E0C3CF10ED180F1A3008F03ACFE1E05D
:101C8000F0E0EC0FFD1F24E0029FE00DF11D112498
:101C90002081318142815381AAE0B0E00E94C024BA
:101CA000610F711D811D911D6083718382839383F8
:101CB00020CF49885A886B887C88812C912C5401CC
:101CC00018CF81149104A104B10489F4C301B201B5
:101CD0000E94930561E070E080E090E00E94531A5A
:101CE0001D8A1E8A1F8A188E312C22242A948D8DDB
:101CF0009E8DAF8DB8A188169906AA06BB06D0F4B2
:101D00000E944D052D893E894F89588D280F311D20
:101D1000411D511D2D8B3E8B4F8B588F381608F46B
:101D2000382E821508F4282E3FEF831A930AA30A4F
:101D3000B30A56C0C301B20128EE33E040E050E0E0
:101D40000E94F724BA01A9012AE030E086E094E07D
:101D50000E94E61D6CE286E094E00E940A1D4AE0C3
:101D600050E0632D86E094E00E94F51D6CE286E071
:101D700094E00E940A1D6D897E898F89988DA50146
:101D800094010E94F724BA01A9012AE030E086E01C
:101D900094E00E94E61D6CE286E094E00E940A1D39
:101DA0004AE050E0622D86E094E00E94F51D6CE26E
:101DB00086E094E00E944A1D4C0C5D1C6E1C7F1C4A
:101DC000898D9A8DAB8DBC8D84159505A605B705BB
:101DD00020F449885A886B887C88812C912C540186
:101DE00029893A894B895C89283E33404105510550
:101DF00009F07FCEA296E2E10C945425ACE1B0E06C
:101E0000E4E0FFE00C9442250E94301A6B017C0153
:101E100081E00E94030614E703E0198361E0CE012C
:101E200001960E94600700939B030E94DE066AEF02
:101E300070E080E090E00E94531A80919B03833011
:101E400089F486E094E00E949D1B892B59F40E943E
:101E5000301A6C197D098E099F096038734C894CC2
:101E60009140D8F280919B03833009F44FC08FE7F3
:101E70000E94FC040E940F058983843511F083E0E1
:101E80005CC00E940F0510926E0380936F030E9446
:101E90000F0520916E0330916F03280F311D309391
:101EA0006F0320936E030E940F05809370030E94BE
:101EB0000F0580937103813110F7F12C0F2D10E085
:101EC0008091710390E0880F991F0817190740F45B
:101ED0000E940F05F801EE58FC4F8083F394EECF7B
:101EE00080E7898361E0CE0101960E94600783E06C
:101EF00080939B030E94DE0662E370E080E090E046
:101F00000E94531A80919B03833011F482E015C024
:101F10008FE70E94FC040E940F058983803509F039
:101F2000AECF07EC13E00E940F05F80181938F01FB
:101F3000F3E0023E1F07B9F781E06C96E8E00C94ED
:101F40005E25CF93C82F682F86E094E00E940E1C78
:101F5000909192039C2790939203CF910895A1E0D2
:101F6000B0E0E5EBFFE00C94482599830E94A10FB7
:101F70009981892F0E94A10F2196E2E00C9464259B
:101F80001F93CF93DF93182FEB011092920365EB11
:101F900086E094E00E940E1C62E686E094E00E94D7
:101FA0000E1C812F0E94A10FCE010E94AF0FDF9166
:101FB000CF911F9108956091920386E094E00E9472
:101FC0000E1C0895A1E2B0E0E8EEFFE00C94442579
:101FD0007B018A018C3009F452C108F040C0863080
:101FE00009F4BCC018F5833009F491C070F4813055
:101FF00009F472C0823009F047C26BE170E082E000
:102000000E94C00F07EC13E078C0843009F487C049
:10201000853009F039C26091710370E0660F771F57
:1020200085E00E94C00F02E713E086C0893009F402
:10203000A7C070F4873009F49BC0883009F024C22F
:1020400061E070E088E00E94C00F8091FC0322C232
:102050008A3009F4CAC08B3009F4F1C015C28A363F
:1020600009F474C1D8F4873609F439C138F48536D7
:1020700009F40DC1863609F41EC106C2883609F47A
:1020800036C1893609F000C261E070E089E60E943D
:10209000C00F0E94EA010E942F02F4C18D3609F49C
:1020A000D3C138F48B3609F490C18C3609F499C148
:1020B000EBC18E3609F4DBC1873C09F0E5C161E074
:1020C00070E087EC0E94C00F81E00E94A10F0E9487
:1020D000DB0F10929303E2C169E270E081E00E949D
:1020E000C00F0EE913E0F80181918F010E94A10F4A
:1020F000F3E0073C1F07B9F7CFC1F80181918F01C9
:102100000E94A10FF3E0023E1F07B9F7C5C161E0CD
:1021100070E083E00E94C00F0E94FE0EBBC161E030
:1021200070E084E00E94C00F81E00E94A10F0E9435
:10213000DB0F0E94310DB2C18091710390E0880FD6
:10214000991F9801225733402817390708F0A4C176
:10215000F80181918F010E94A10FEECF62E070E043
:1021600086E00E94C00F80E893E00E94AF0F94C108
:1021700061E070E087E00E94C00F809170038AC127
:1021800086E6898361E0CE0101960E9460070E9485
:10219000DE0683E080939B0368EC70E080E090E0D3
:1021A0000E94531A80919B038430D9F48FE70E94D8
:1021B000FC040E940F058983863469F460E270E0B4
:1021C00089E00E94C00F10E20E940F050E94A10F3B
:1021D0001150D1F761C161E070E089E00E94C00F49
:1021E00051C161E070E089E052C169E170E08AE0CC
:1021F0000E94C00F1092E20320919A038091E7039E
:102200009091E803A091E903B091EA03222311F031
:10221000806801C08F778093E7039093E803A093D1
:10222000E903B093EA0302EE13E0F80181918F0114
:102230000E94A10FF3E00B3F1F07B9F72DC161E228
:1022400070E08BE00E94C00F80913A038F3F39F01D
:1022500080913A0391E0980F90933A0302C08091E5
:102260003A030E94A10F10E0812F0E940C0D0E94E2
:102270008D040E94AF0F1F5F1031B1F70DC161E0F7
:1022800070E08CE00E94C00F8091FB0303C161E00D
:1022900070E085E60E94C00F89E2E816F10409F0BB
:1022A000F8C0D801EEE9F3E08D91819383E0E73C3B
:1022B000F807D1F7E7C061E070E086E60E94C00F42
:1022C000EBE1EE16F10409F0E4C0D801E7ECF3E02D
:1022D0008D91819383E0E23EF807D1F7D3C061E0AE
:1022E00070E087E60E94C00F0E94B708CBC061E093
:1022F00070E088E60E94C00F85E789838BE1E7ECF8
:10230000F3E0DE01129601900D928A95E1F76CE1FF
:10231000CE0101960E9460070E94DE0683E0809352
:102320009B0360E273E080E090E00E94531A80918A
:102330009B03843009F0ADC08FE70E94FC040E942B
:102340000F058983853509F0A4C09CC061E070E069
:102350008AE60E94C00F89E6898361E0CE0101967A
:102360000E9460070E94DE0683E080939B0360E288
:1023700073E080E090E00E94531A80919B038430C8
:1023800009F087C08FE70E94FC040E940F05898333
:102390008E010E5F1F4F7E01EDE1EE0EF11C0E94DB
:1023A0000F05F80181938F01EE15FF05C1F78BE151
:1023B000FE013296A7ECB3E001900D928A95E1F709
:1023C0008981893409F065C05DC061E070E08BE609
:1023D0000E94C00FF80180818093FC030E94C00816
:1023E00051C061E070E08CE60E94C00FF0E2EF1691
:1023F000F10461F487E6898380E2F801DE01129638
:1024000001900D928A95E1F761E203C087E4898328
:1024100061E0CE0101960E9460070E94DE0683E023
:1024200080939B036CE474E080E090E00E94531A78
:1024300080919B03843069F58FE70E94FC040E9421
:102440000F05873431F51EC061E070E08DE60E9413
:10245000C00F89E1E816F104E1F4D801E2EEF3E0FF
:102460008D91819383E0EB3FF807D1F70BC061E0DA
:1024700070E08EE60E94C00FF80180818093FB031C
:102480000E94A00881E006C061E070E08AEC0E9432
:10249000C00F80E00E94A10F0E94DB0FA196E6E032
:1024A0000C946025A0E0B0E0E8E5F2E10C94422550
:1024B000CAE5D2E014E606E035E0F32E44E0E42E6F
:1024C00053E0D52E62E0C62E86E094E00E949D1B6C
:1024D000892B09F49BC086E094E00E94C11B282F41
:1024E0008093C5024091C40250E04730510560F727
:1024F000FA01EA5AFF4F0C946F25853B29F781E0DA
:102500008093C402E1CF823609F07DC0C092C4023C
:10251000DBCF8093C3028093C202D092C402D4CF97
:102520009C0133273093C1022093C0029091C202D4
:1025300098279093C202E092C402C6CF382F222778
:102540004091C0025091C102242B352B3093C1021F
:102550002093C0029091C20298279093C202F092F9
:10256000C4022536310508F4AFCF61E070E08CEC91
:102570000E94C00F81E00E94A10F0E94DB0F43C0A8
:102580002091BE023091BF02F901E65AFD4F8083CF
:102590009091C20298279093C202C901019690932C
:1025A000BF028093BE022091C0023091C102821707
:1025B000930708F489CF0093C40286CF8091C202AA
:1025C00082130BC06091BE027091BF024AE552E0D7
:1025D0008091C3020E94E20F0DC062E070E08BECBC
:1025E0000E94C00F8091C3020E94A10F80919203AC
:1025F0000E94A10FFE01812F11928A95E9F7109296
:10260000BF021092BE021092C4025ECFCDB7DEB7F9
:10261000E8E00C945E2581E080939303809193031E
:10262000882349F086E094E00E949D1B892BB1F33A
:102630000E945212F3CF0895AAE2B0E0E2E2F3E181
:102640000C9440250E94241A6B017C0181E00E94B9
:10265000030686E094E00E949D1B892B29F086E00A
:1026600094E00E94C11BF5CF5F9811E072E6B72E8F
:10267000E9E2AE2E03E00E94241A6C197D098E094E
:102680009F09693C710581059105D0F11123C1F1C4
:102690000E94241A6B017C01469A80ED97E00E940B
:1026A000FF02B982EEE9F3E0DE0112968A2D019075
:1026B0000D928A95E1F76AE2CE0101960E946007C9
:1026C000469880E090E00E94FF0200939B030E94E6
:1026D000DE0662E370E080E090E00E94531A809191
:1026E0009B03843061F400939B038FE70E94FC04FA
:1026F0000E940F0511E0823419F410E001C011E0CE
:1027000082E10E94741B892B81F411E00EC05F9A54
:10271000469A86E094E00E94C11B8D309105A9F095
:102720005CF40A9791F05F98469886E094E00E94E6
:102730009D1B892B61F79FCF8332910569F082340D
:10274000910589F70E940B13EECF66ED70E086E0ED
:1027500094E00E94261DE7CF0E94310DE4CF8F92B6
:102760009F92AF92BF92CF92DF92EF92FF921F9310
:10277000CF93DF9382E10E94741B892B09F089C0FB
:1027800068EC70E080E090E00E94531A80E090E0F6
:102790000E94FF020E94241A4B015C016B017C0124
:1027A00080ECC80E82E1D81EE11CF11C0E94241AA4
:1027B0006C157D058E059F0530F482E10E94741B27
:1027C000892BA1F364C082E10E94741B892B09F05C
:1027D0005EC080ED97E00E94FF020E94241A6B0108
:1027E0007C01D0E0C1E088E4880E86E2981EA11C3E
:1027F000B11C11E082E10E94741B892B21F58C141D
:102800009D04AE04BF0430F480ED97E00E94FF0207
:10281000D1E0F0CF0E94241A6C197D098E099F091E
:10282000693C71058105910528F30E94241A6B010A
:102830007C01C12719F080ED97E002C080E090E0B4
:102840000E94FF02D7CF80E090E00E94FF02DD23CC
:10285000B9F08091FB0390E0019665E070E00E9482
:10286000E3248093FB030E94A0080E94010B0E94B6
:10287000C00864EF71E080E090E00E94531A09C044
:1028800080E00E944F020E941E090E94B7080E9429
:102890001C13DF91CF911F91FF90EF90DF90CF90AD
:1028A000BF90AF909F908F900895CF92DF92EF925C
:1028B000FF9280E00E945C030E94200361E086E0BA
:1028C0000E94081B61E085E00E94081B60E082E135
:1028D0000E94081B60E084E00E94081B61E084E025
:1028E0000E94411B0E94F30260E070E086E094E0E9
:1028F0000E94931C0E94010B0E94C0080E94E60ADD
:102900008FEF80933A030E942C0378940E94241A3C
:102910006B017C0180913A038F3F59F40E94241A85
:102920006C197D098E099F09603D774081059105ED
:1029300088F380ED97E00E94FF0261E082E10E944F
:10294000411B5F9A86E094E00E949D1B892B29F031
:1029500086E094E00E94C11BF5CF6EEE71E086E048
:1029600094E00E94071D80E893E00E94B50765E0AF
:1029700072E086E094E00E94071D4AE050E066E0C5
:1029800070E086E094E00E94CE1D62E370E080E09B
:1029900090E00E94531A86E094E00E949D1B0497E9
:1029A0000CF186E094E00E94C11B82349105D1F4C1
:1029B00086E094E00E94C11B8E34910599F486E074
:1029C00094E00E94C11B8434910561F486E094E098
:1029D0000E94C11B819731F480E090E00E94FF02C9
:1029E0000E941C1340919F035091A0036091A1038A
:1029F0007091A203DB01CA010197A109B1090497F3
:102A0000A105B10568F440933903433029F440EA45
:102A100056E861E070E004C040E052EC61E070E034
:102A200088E594E00E94631F0E94AF135F9880E0E6
:102A300090E00E94FF020E94E60A109255038091E6
:102A4000E70383FF11C08091B303882351F0809185
:102A5000BA03882331F08091C103882311F087E005
:102A600001C085E08093550380E00E9403068091B9
:102A700056030E9437050E94DE061092CF02109284
:102A8000CE021092CD02F12C8091FC038F15B0F094
:102A900062E370E080E090E00E94531A80ED97E0DE
:102AA0000E94FF0262E370E080E090E00E94531A0F
:102AB00080E090E00E94FF02F394E6CF8091C6038D
:102AC00084FF08C0982F987181E0983109F080E068
:102AD0000E94DA088FE00E945C03FF90EF90DF9085
:102AE000CF900895EF92FF920F931F93CF93DF93B0
:102AF0008C016EE770E088E594E00E94C901E8016E
:102B0000F12CF0E2EF2E8E0188818D57823048F44F
:102B10006DE770E088E594E00E94C90188818E2508
:102B200088832196F801608188E594E00E94751EF3
:102B3000F394F9E0FF12E7CF6EE770E088E594E0E8
:102B40000E94C901CDB7DEB7E6E00C946025A9E08C
:102B5000B0E0EDEAF5E10C9448259091570391110E
:102B60000EC09EEF99838A836B8350E055954795FD
:102B70004C832D83198618861F821E822EC0409199
:102B80005C03842F90E0B4E095958795BA95E1F7C2
:102B9000242F2F7030E08217930719F18DEF89836E
:102BA0001B82FE01349650E0842F90E0A4E09595BE
:102BB0008795AA95E1F7242F2F7030E082179307AD
:102BC00049F0DC01A35ABC4F8C918193405F5F5F59
:102BD000563051F740935C035A83CE0101960E9410
:102BE00072158091570390E0019666E070E00E94B4
:102BF000E324809357032996E2E00C946425A0E037
:102C0000B0E0E5E0F6E10C9441256C016EE770E080
:102C100088E594E00E94C9018601E12CF12CC0E016
:102C2000D0E030E2B32EF801608183E8860F823075
:102C300078F46DE770E088E594E00E94C901F8013E
:102C400060816B2570E088E594E00E94C90104C0B2
:102C500088E594E00E94751EE114F10459F0F80132
:102C600080819E01280F311DC901C92FDD27C80FA2
:102C7000D91FDD273FEFE31AF30A89E0E816F104D4
:102C800059F028E0E216F10421F48C2F8095F6012A
:102C900080870F5F1F4FC7CFCDB7DEB7E9E00C9439
:102CA0005D25A9E0B0E0E7E5F6E10C944825E82FC2
:102CB000362F8091570390E0019664E270E00E9405
:102CC000E3248093570358E9598350E15A838130B4
:102CD00089F048F08230B9F08330D9F48B8381EFEA
:102CE0008C833D8319C085E08B8381EF8C832F5FBC
:102CF0002D8312C08B8381EF8C8384E6489FA001D3
:102D000011245D8309C084E08B8381EF8C83ED8384
:102D100003C00E94170904C0CE0101960E94FF154E
:102D20002996E2E00C946425A2E0B0E0EAE9F6E13D
:102D30000C943D25182F762E2A8349830E94301A41
:102D40006B017C0180916D03809058039090590332
:102D5000A0905A03B0905B032A8149818823C1F077
:102D6000D701C60188199909AA09BB094C015D015F
:102D700091EE89169EE29906A104B10420F1241770
:102D800008F4422F202F672D812F0E94511613C067
:102D9000D701C60188199909AA09BB094C015D012F
:102DA00091E3891695E79906A104B10460F0672DB7
:102DB000812F0E94A715C0925803D0925903E09228
:102DC0005A03F0925B032296EDE00C945925A2E29F
:102DD000B0E0EDEEF6E10C943E258CE00E941E057D
:102DE00081110DC06DE072E086E094E00E94381D14
:102DF0005F9A80E00E9403060E94DE065F9888E5E5
:102E000094E00E941B1E892B01F188E594E00E944A
:102E1000481E90913903992319F00E94140BEFCFAB
:102E20004091CE0250E09A012F5F3F4F2F71332720
:102E30006091CF0270E02617370709F3FA01E752D5
:102E4000FD4F80832093CE02DACF80913903811128
:102E500006C080919B03843009F094C00DC086E0C9
:102E600094E00E949D1B892BA1F386E094E00E94D0
:102E7000C11B0E94140BF3CF0E94301A611571051B
:102E80008105910549F0609347037093480380934F
:102E9000490390934A030CC081E090E0A0E0B0E0C9
:102EA0008093470390934803A0934903B0934A0348
:102EB00080913D0390913E03816090933E03809307
:102EC0003D0383E080939B038FE70E94FC0409EF9E
:102ED00012E00E940F05F80181938F01F3E00230A8
:102EE0001F07B9F7209102038091F902982F9227CA
:102EF00096FF3BC090E4922790930203982F98731B
:102F00009833F1F410E0212F30E08091F9028770BE
:102F100090E0821793074CF11F5F2091C603812F29
:102F200090E0FC01E750FD4F24FF04C080810E9427
:102F3000F908E9CF608188E594E00E94751EE3CF2F
:102F40008F7399F48091FA02809346038091FB027B
:102F5000809344038091FC02809343038091FF029D
:102F600090E090933C0380933B038091CD028130AD
:102F700019F482E08093CD028091CD02833011F468
:102F80001092CD020E94301A6B017C0180913F03A8
:102F900090914003A0914103B09142030097A10595
:102FA000B105C9F0A7019601281B390B4A0B5B0B31
:102FB000DA01C901883B9B40A105B10560F00E9480
:102FC0004D058093450310923F03109240031092E9
:102FD00041031092420380914B0390914C03A091C6
:102FE0004D03B0914E0346015701881A990AAA0A67
:102FF000BB0A8EE993E00E94780386169706A8061E
:10300000B90608F4A8C0C0924B03D0924C03E092DA
:103010004D03F0924E030E94C00180913A03883024
:10302000A0F08091E7039091E803A091E903B091AB
:10303000EA036CE1B695A795979587956A95D1F7C0
:10304000892B8A2B8B2B09F0A4C180913A038F5FC7
:1030500080933A038091470390914803A0914903DC
:10306000B0914A030097A105B105F1F0C81AD90A39
:10307000EA0AFB0A8EE993E00E9478036C157D054D
:103080008E059F0508F006C18091E70384FD04C00A
:1030900080ED97E00E94FF021092470310924803D0
:1030A0001092490310924A0390910203907C9093EE
:1030B00002035091CE028091CF022091CD02581789
:1030C00009F405C1223009F002C19058909302031F
:1030D000E091C603E770F0E0E45EFD4F6081693087
:1030E00008F0DDC0615040E04613DBC08093CF02A2
:1030F00087E3840F90910203892B8093020340930E
:10310000D00283E08093CD02469A8091AB039091E8
:10311000550391112FC10E94FE05809156030E9414
:103120003705E091C603E770F0E0E45EFD4F608193
:1031300082E093E00E941907E0915603EF5FE0936D
:103140005603E83109F422C1F0E0E256FC4F8785CE
:10315000882309F41BC10E948807813069F580919A
:10316000C603887149F180913D0390913E03880F19
:10317000991F90933E0380933D0383E080939B03CC
:103180000E94DE060E94301A60933F037093400352
:103190008093410390934203672B682B692B61F462
:1031A00081E090E0A0E0B0E080933F039093400383
:1031B000A0934103B09342038091C60384FF1FC0D4
:1031C00080913D0390913E038E7F0E94AE04182FA4
:1031D00060913B03809146030E940A0B482F612FA8
:1031E0008091450349A30E940A0B0091FC03282FFC
:1031F00049A160914303809144030E94941646982C
:10320000809153038130C1F018F08230B1F1CEC00B
:1032100082E10E94741B892B09F0C8C081E0809371
:1032200053030E94241A60934F03709350038093BA
:10323000510390935203BAC082E10E94741B892B00
:1032400031F50E94241AC0904F03D0905003E090B3
:103250005103F09052036C197D098E099F09693E54
:1032600073408105910508F4A1C082E08093530367
:1032700080ED97E00E94FF0299C082E10E94741BDA
:10328000892B09F493C080E090E00E94FF02109225
:1032900053038CC080E090E00E94FF0205CF68E0FD
:1032A00022CF851709F422CF4F5F242F30E090E022
:1032B000F901EE5FFC4FDC01A752BD4F7C9170839A
:1032C000F901E053FD4F708301968F710DCF2430CB
:1032D000B1F42091D00281ED92E0A3E0B3E0FC01D3
:1032E0003E2F381B321718F431913D93F9CF87E305
:1032F000820F90910203892B8093020302CF809169
:103300005303823069F49160909302035F9A5BEEFD
:10331000E52E53E0F52E8E010F5F1F4FB80110C050
:103320005F988091CD02811103C081E08093CD022E
:103330008091CD02833059F784E08093CD02E7CFAE
:10334000F70181917F0169A37AA30E940C0DF80116
:10335000819391938F0169A17AA1FBEFEF16F3E0BE
:10336000FF0671F78091C60343E053E087700E9427
:10337000FD03CACE882309F4CECE2091540331E058
:10338000320F309354032913C6CE0CC0109256034B
:10339000E2CE80913A03883009F45F9A89E0809305
:1033A0003A03D9CE109254038150B5CEA296ECE0E8
:1033B0000C945A251F920F920FB60F9211242F933F
:1033C0003F938F939F93AF93BF938091FE03909110
:1033D000FF03A0910004B09101043091FD0323E0AC
:1033E000230F2D3720F40196A11DB11D05C026E83D
:1033F000230F0296A11DB11D2093FD038093FE03B0
:103400009093FF03A0930004B09301048091020401
:1034100090910304A0910404B09105040196A11DAC
:10342000B11D8093020490930304A0930404B0930D
:103430000504BF91AF919F918F913F912F910F9074
:103440000FBE0F901F9018952FB7F8946091FE0350
:103450007091FF0380910004909101042FBF0895A3
:103460003FB7F8948091020490910304A091040462
:10347000B091050426B5A89B05C02F3F19F0019611
:10348000A11DB11D3FBF6627782F892F9A2F620F8C
:10349000711D811D911D42E0660F771F881F991FC6
:1034A0004A95D1F70895CF92DF92EF92FF92CF9392
:1034B000DF936B017C010E94301AEB01C114D1042F
:1034C000E104F10479F00E94301A6C1B7D0B683E18
:1034D0007340A0F381E0C81AD108E108F108C8518F
:1034E000DC4FECCFDF91CF91FF90EF90DF90CF904A
:1034F0000895789484B5826084BD84B5816084BD6C
:1035000085B5826085BD85B5816085BDEEE6F0E05C
:10351000808181608083E1E8F0E0108280818260B8
:103520008083808181608083E0E8F0E08081816039
:103530008083E1E9F0E08081826080838081816026
:103540008083E0E9F0E0808181608083E1ECF0E05D
:1035500080818460808380818260808380818160BB
:103560008083E3ECF0E0808181608083E0ECF0E038
:10357000808182608083E2ECF0E0808181608083E2
:10358000EAE7F0E0808184608083808182608083CC
:10359000808181608083808180688083089590E04D
:1035A000FC013197EE30F10590F5E35AFF4F0C9492
:1035B0006F25809180008F7703C0809180008F7D80
:1035C00080938000089584B58F7702C084B58F7D85
:1035D00084BD0895809190008F7707C080919000FE
:1035E0008F7D03C080919000877F80939000089525
:1035F0008091C0008F7703C08091C0008F7D809341
:10360000C00008958091C200877F8093C200089512
:10361000CF93DF9390E0FC01E75EFE4F2491FC0125
:10362000E95CFE4F8491882349F190E0880F991F4F
:10363000FC01EF58FE4FA591B4918D599E4FFC01AE
:10364000C591D4919FB7611108C0F8948C912095D1
:1036500082238C93888182230AC0623051F4F894CB
:103660008C91322F309583238C938881822B888391
:1036700004C0F8948C91822B8C939FBFDF91CF91E3
:103680000895A1E0B0E0E7E4FBE10C944625282F83
:1036900030E0F901E550FF4F8491F901E75EFE4FFC
:1036A0001491F901E95CFE4F04910023C9F08823CD
:1036B00021F069830E94CF1A6981E02FF0E0EE0FBC
:1036C000FF1FED59FE4FA591B4919FB7F8948C91CF
:1036D000611103C01095812301C0812B8C939FBF82
:1036E0002196E4E00C946225CF93DF93282F30E0FD
:1036F000F901E550FF4F8491F901E75EFE4FD49147
:10370000F901E95CFE4FC491CC2391F081110E9434
:10371000CF1AEC2FF0E0EE0FFF1FEB5AFE4FA591F2
:10372000B4912C912D2381E090E021F480E002C03F
:1037300080E090E0DF91CF910895809154049091C2
:1037400055042091560430915704821B930B8F73BC
:10375000992708952091540430915504809156047E
:10376000909157042817390749F0E0915604F091D9
:103770005704EC5EFB4F808190E008958FEF9FEF40
:1037800008952091540430915504809156049091ED
:10379000570428173907A9F0E0915604F09157040F
:1037A000EC5EFB4F808120915604309157042F5FCF
:1037B0003F4F2F733327309357042093560490E0E4
:1037C00008958FEF9FEF0895CF93DF93C091540436
:1037D000D09155042196CF73DD27809156049091A6
:1037E0005704C817D90799F082E00E9499208F3FAB
:1037F0002FEF920761F0E0915404F0915504EC5ED4
:10380000FB4F8083D0935504C0935404DFCFDF91E6
:10381000CF91089583E00E94E4220895A1E0B0E0F2
:10382000E4E1FCE10C9446258C0169838091A401BC
:10383000882359F041E050E0BE016F5F7F4F83E085
:103840000E94CC20181619063CF081E090E0F801A7
:103850009383828380E090E02196E4E00C946225DB
:10386000FC0120812E5F208342E450E06FE771E08D
:1038700080E80E944C210895FC0181819081913A59
:1038800059F4813209F04BC047E050E06DE971E036
:1038900080E00E944C2145C0913209F040C0803246
:1038A00039F467E070E08DE991E00E94902139C021
:1038B000823209F034C082818093A40180919D01FD
:1038C00090919E01A0919F01B091A001803B9440F6
:1038D000A105B10531F58091A40180FD12C087E7F3
:1038E00097E790930108809300082BE088E190E02F
:1038F0000FB6F894A895809360000FBE20936000E7
:1039000010C088E10FB6F8948093600010926000B8
:103910000FBEA895109201081092000802C080E026
:10392000089581E008950895109209041092080402
:1039300088EE93E0A0E0B0E080930A0490930B043B
:10394000A0930C04B0930D048EE292E090930704D0
:10395000809306040895A0E0B0E0E1EBFCE10C9454
:1039600042256C017A01EB01E60EF71E00E010E043
:10397000CE15DF0561F06991D601ED91FC910190C2
:10398000F081E02DC6010995080F191FF1CFC8017C
:10399000CDB7DEB7E8E00C945E256115710589F0BE
:1039A000DB010D900020E9F7AD0141505109461BA4
:1039B000570BDC01ED91FC910280F381E02D09951C
:1039C000089580E090E00895EF92FF920F931F9387
:1039D000CF93DF938C01FB01C0E0D0E064917F01C5
:1039E0008FEFE81AF80A662361F0D801ED91FC9197
:1039F0000190F081E02DC8010995C80FD91FF7018A
:103A0000EDCFCE01CDB7DEB7E6E00C9460250E9485
:103A1000CD1C0895DC01ED91FC910190F081E02D29
:103A2000099508950F931F93CF93DF93EC016DE0F9
:103A30000E940A1D8C016AE0CE010E940A1D800FBF
:103A4000911FDF91CF911F910F9108950F931F93B5
:103A5000CF93DF93EC010E94E41C8C01CE010E9405
:103A6000121D800F911FDF91CF911F910F9108952B
:103A70000F931F93CF93DF93EC010E94CD1C8C0119
:103A8000CE010E94121D800F911FDF91CF911F91D7
:103A90000F9108950F931F93CF93DF93EC010E9432
:103AA0000A1D8C01CE010E94121D800F911FDF9113
:103AB000CF911F910F910895A1E2B0E0E2E6FDE100
:103AC0000C943E257C01C42EE52FCB01D22E19A2E9
:103AD00021E02D1510F02AE0D22E8E010F5D1F4F30
:103AE0008D2C912CA12CB12C6C2D7E2FA501940135
:103AF0000E94F7248C2DD29E8019112401501109A7
:103B00008A3010F4805D01C0895CF8018083211542
:103B100031054105510521F0C22EE32FCA01E4CF42
:103B2000B801C7010E94CD1CA196ECE00C945A2567
:103B3000A0E0B0E0EEE9FDE10C944225EC016A0161
:103B40007B012115310541F4E881F9810190F08173
:103B5000E02D642F09951DC02A303105A9F477FFA7
:103B600012C06DE20E940A1D8C0144275527BA013C
:103B70004C195D096E097F092AE0CE010E945C1D87
:103B8000800F911F06C02AE0B701A601CE010E9456
:103B90005C1DCDB7DEB7E8E00C945E250F931F9354
:103BA000CF93DF93EC019A01AB01662757FD609537
:103BB000762F0E94981D8C01CE010E94121D800F4D
:103BC000911FDF91CF911F910F910895211531051C
:103BD00049F4DC01ED91FC910190F081E02D642F1E
:103BE000099508950E945C1D08959A01462F50E0A2
:103BF00060E070E00E94E61D08959A01AB0160E06C
:103C000070E00E94E61D08950F931F93CF93DF93FA
:103C1000EC019A01462F50E060E070E00E94E61D42
:103C20008C01CE010E94121D800F911FDF91CF9158
:103C30001F910F910895FC0124853585F901E05C01
:103C4000FF4F80819181F901EE5BFF4F208131812F
:103C5000821B930B8F7399270895FC0184859585AA
:103C6000FC01E05CFF4F40815181FC01EE5BFF4FA6
:103C7000208131814217530741F00190F081E02DFE
:103C8000E80FF91F808190E008958FEF9FEF08956E
:103C9000FC0184859585FC01E05CFF4F40815181EA
:103CA000FC01EE5BFF4F208131814217530779F011
:103CB000A081B181A80FB91F8C91208131812F5F24
:103CC0003F4F2F7333273183208390E008958FEF88
:103CD0009FEF0895FC0181A1882329F0A489B5896B
:103CE0008C9186FFFBCF11A20895CF93DF93FC0147
:103CF00026853785D901A05CBF4F8D919C91119786
:103D000001968F739927E901CE5BDF4F4881598176
:103D100084179507D9F30D90BC91A02DA20FB31F66
:103D20006C93A685B785A05CBF4F11969C938E932C
:103D3000A689B7892C9181E090E0078C02C0880F9A
:103D4000991F0A94E2F7282B2C9381E081A3048821
:103D5000F589E02D80818064808381E090E0DF91AF
:103D6000CF91089508951F920F920FB60F921124CC
:103D70002F933F934F938F939F93EF93FF93809154
:103D8000C80082FD1CC04091CE008091FE0490913D
:103D9000FF0401968F73992720910005309101054A
:103DA0008217930771F0E091FE04F091FF04E25452
:103DB000FB4F40839093FF048093FE0402C08091E8
:103DC000CE00FF91EF919F918F914F913F912F9155
:103DD0000F900FBE0F901F90189588E594E00E94F9
:103DE0001B1E892B11F00E94B21E08951F920F9284
:103DF0000FB60F9211242F933F938F939F93EF93BE
:103E0000FF932091BA043091BB048091BC0490913F
:103E1000BD042817390731F48091C9008F7D809344
:103E2000C90014C0E091BC04F091BD04E658FB4FFA
:103E300020818091BC049091BD0401968F739927D5
:103E40009093BD048093BC042093CE00FF91EF912A
:103E50009F918F913F912F910F900FBE0F901F90C8
:103E60001895A0E0B0E0E7E3FFE10C943E25FC01EB
:103E70001382128288EE93E0A0E0B0E08483958301
:103E8000A683B78380E492E09183808375876487FB
:103E900057874687318B208B138B028BF58AE48AF8
:103EA000D78AC68AB18EA08E938E828E8F85848F9C
:103EB0008889858F8989868F8A89878F8B8980A356
:103EC000ECE00C945A25CF92DF92EF92FF92CF93C1
:103ED000DF93EC016A017B01411581EE5807610512
:103EE0007105F9F0EC89FD8981E090E008A002C03D
:103EF000880F991F0A94E2F7808360E079E08DE3F0
:103F000090E0A70196010E94F72421503109410950
:103F100051095695479537952795211580E1380722
:103F200098F0EC89FD89108260E874E88EE190E0F9
:103F3000A70196010E94F724215031094109510936
:103F40005695479537952795E889F9893083EA8909
:103F5000FB89208319A2EE89FF89408181E090E0EE
:103F60009C010C8C02C0220F331F0A94E2F7422BF3
:103F70004083EE89FF8940819C010D8C02C0220F95
:103F8000331F0A94E2F7422B4083EE89FF89408178
:103F90009C010E8C02C0220F331F0A94E2F7422BC1
:103FA0004083EE89FF8920810F8C02C0880F991F02
:103FB0000A94E2F7809582238083DF91CF91FF906E
:103FC000EF90DF90CF9008958F929F92AF92BF9223
:103FD000CF92DF92EF92FF920F931F9381E08F9326
:103FE00085E08F9387E08F9383E08F9384E08F93B6
:103FF000EEEC8E2E912CFAECAF2EB12CA9ECCA2E41
:10400000D12CB8ECEB2EF12C0CEC10E02DEC30E0C8
:104010004AE754E06EEB74E088E594E00E94311FBB
:104020000F900F900F900F900F901F910F91FF9096
:10403000EF90DF90CF90BF90AF909F908F900895BA
:104040000E94791A82E095E00E94EE220E945514A7
:10405000CDEEDEE10E94E7162097E1F30E94ED1E0F
:10406000F9CF615030F02091F100FC0120830196DE
:10407000F8CF289884E68093090508952FB7FC01AE
:104080002083F89467706093E9000895A1E0B0E0A0
:10409000ECE4F0E20C944825682FCE0101960E94D2
:1040A0003E208091F20099819FBF2196E2E00C941E
:1040B0006425A2E0B0E0EFE5F0E20C944525F62E91
:1040C0008A0190910805992311F057FF03C08FEFE3
:1040D0009FEF2BC0682FCE0101967A830E943E206D
:1040E0008091F20090E0A8017A81801791070CF48A
:1040F000AC01EF2DF72FF40E84E6FE1639F0289868
:10410000809309059091F1009193F7CF41155105E6
:1041100021F08091F200882321F089818FBFCA01AC
:1041200004C08BE68093E800F8CF2296E5E00C947B
:104130006125A1E0B0E0EFE9F0E20C94482541E010
:1041400050E0BE016F5F7F4F0E945920019719F424
:10415000898190E002C08FEF9FEF2196E2E00C94FE
:104160006425A1E0B0E0E7EBF0E20C944825682F6D
:10417000CE0101960E943E209091E800892F807226
:1041800095FF04C09091F20080E4891B99819FBF44
:104190002196E2E00C946425A1E0B0E0E2EDF0E2CB
:1041A0000C943A25582E7B01A42E952E809108055B
:1041B000882369F0042F152F8AEFB82E852D807281
:1041C000782E9AE3892E852D8074682E11C08FEF8A
:1041D0009FEF53C0852D0E94B120482E81110CC045
:1041E000BA94A9F361E070E080E090E00E94531A75
:1041F0000115110579F737C0282F30E00217130792
:104200000CF4402EC42CD12C0C191D09652DCE01A7
:1042100001960E943E20772039F04A948FEF48168D
:10422000B1F01092F100F9CFF701842D57FE07C0CD
:10423000815058F094919093F1003196F9CF8150CC
:1042400020F091919093F100FACFEC0CFD1C80913D
:10425000E80085FF0FC00115110511F461100AC0B7
:1042600089818FBFC5CF5D9884E680930A058A2D2A
:10427000992D03C08092E800F3CF2196E0E10C94E1
:1042800056251092E90010920705109206059093AA
:104290000505809304050895CF93DF93FB0120E08B
:1042A00030E0DEEF24173507A1F187FF02C0C4918B
:1042B00001C0C081A0910605B09107056091040579
:1042C00070910505A617B707B4F49091E8009570B2
:1042D000E1F39091E80092FD1EC0C093F10060915F
:1042E0000605709107056F5F7F4F6F737727672B08
:1042F00011F4D093E80060910605709107056F5F97
:104300007F4F70930705609306052F5F3F4F3196EF
:10431000C9CFC90102C08FEF9FEFDF91CF91089500
:10432000A1E0B0E0E6E9F1E20C944725162F2091D8
:10433000E80022FFFCCF612F79830E9431208BEFB0
:104340008093E800812F7981972F2196E3E00C94E8
:104350006325A1E0B0E0EFEAF1E20C944825198270
:10436000CE0101960E94301CCE0101960E94882346
:10437000898190E02196E2E00C9464251F920F92CF
:104380000FB60F921124EF92FF920F931F932F936A
:104390003F934F935F936F937F938F939F93AF93CD
:1043A000BF93EF93FF93CF93DF93CDB7DEB76297C1
:1043B000DEBFCDBF1092E9008091E80083FFE7C027
:1043C00068E0CE010A960E94312082EF8093E800D7
:1043D0009A8597FF05C08091E80080FFFCCF03C05D
:1043E0008EEF8093E800892F807609F0B5C08B8529
:1043F000811105C01092F1001092F100C1C0282F68
:104400002D7F213009F4BCC0853049F48091E8004B
:1044100080FFFCCF8C8580688093E300B1C086303C
:1044200009F072C02D85E888F988223071F580E0A6
:1044300090E02A8B0E9441210E94A92199E08E01DF
:104440000F5F1F4FF801392F11923A95E9F79983C1
:104450002A892A8391E09E8390E898879AEF99872A
:104460002091060530910705275F3F4F3C832B8342
:104470008D83C7010E94412149E050E0B80180E0EE
:104480000E944C210E94A9217BC0C7012A8B0E9457
:1044900041212A89223241F482E290E00E94942351
:1044A000892B09F06DC070C0213069F48889998921
:1044B000089711F42093030580910305882389F060
:1044C00066EC71E016C0233009F05EC08C8588234D
:1044D00059F0823061F0813009F056C06AEE71E027
:1044E00008C068ED71E005C064E272E002C062E0FD
:1044F00072E06115710509F447C0FB01449150E079
:1045000080E80E944C213CC0873009F43DC08830CF
:1045100021F481E08093F10033C0893089F59370F4
:1045200099F5E2ECF1E081E021E096E38093E90087
:104530002093EB0034913093EC009093ED008F5F6B
:104540003196853099F78EE78093EA001092EA0061
:104550008C858093080514C0888999890E9441211F
:104560008E85811105C0CE010A960E943C1C06C0B2
:10457000823051F4CE010A960E94B623882321F09E
:104580008EEF8093E80003C081E28093EB00629697
:104590000FB6F894DEBF0FBECDBFDF91CF91FF9174
:1045A000EF91BF91AF919F918F917F916F915F91AB
:1045B0004F913F912F911F910F91FF90EF900F908E
:1045C0000FBE0F901F9018958093E9008091F20024
:1045D000882319F08AE38093E80008951092080573
:1045E00081E08093D70080EA8093D80082E189BD82
:1045F00009B400FEFDCF61E070E080E090E00E9431
:10460000531A80E98093D8008CE08093E2001092E6
:10461000E000559A209A08951F920F920FB60F92BC
:1046200011242F933F934F935F936F937F938F93B7
:104630009F93AF93BF93EF93FF938091E10010920C
:10464000E10083FF0FC01092E90091E09093EB002E
:104650001092EC0092E39093ED001092080598E020
:104660009093F00082FF26C083E00E94E42282E063
:104670000E944620882321F086E094E00E94E41BFB
:1046800080910A05882339F080910A058150809332
:104690000A05882369F080910905882359F08091E3
:1046A0000905815080930905811104C0289A02C030
:1046B0005D9AF1CFFF91EF91BF91AF919F918F9153
:1046C0007F916F915F914F913F912F910F900FBE0E
:1046D0000F901F901895FF920F931F93CF93DF9326
:1046E000EC01F62EE881F9810480F581E02D099531
:1046F0008C01E881F9810680F781E02D6F2DCE01D4
:104700000995C8019927CDB7DEB7E5E00C9461257E
:10471000FC0120812F5F208349E150E068EA72E0CC
:1047200080E80E944C21089545E650E061EC72E07B
:1047300080E80E944C210895A1E0B0E0E2EAF3E2B3
:104740000C94442589838B017A0141E050E0BE013D
:104750006F5F7F4F84E00E94CC20A701B80184E402
:104760000E94CC202196E6E00C946025FC0191810A
:104770008081813A31F481E0913091F0933089F475
:1047800011C0813271F49B3021F482818093A601A3
:1047900005C09A3031F482818093A50181E00895AB
:1047A000089580E00895FC0110820895FC011382B1
:1047B000128220E532E031832083089548E050E002
:1047C00082E00E949C230895CF93DF93DC01683838
:1047D00018F0E8E7E60F25C0E62FF0E067FF11C00C
:1047E000E058F10981E090E001C0880FEA95EAF70E
:1047F00014969C911497982B14969C931497E0E030
:1048000010C0E85DFD4FE491EE2309F440C0E7FFDE
:1048100008C014968C911497826014968C93149708
:10482000EF7716968C9116978E1741F117968C910B
:1048300017978E1719F118968C9118978E17F1F01B
:1048400019968C9119978E17C9F01A968C911A9710
:104850008E17A1F01B968C911B978E1779F080E034
:1048600090E0ED01C80FD91F2E81211102C0EE8307
:1048700005C0019686309105A1F709C0BD016C5FA6
:104880007F4FCD010E94DE2381E090E008C081E0EF
:1048900090E013969C938E93129780E090E0DF91C6
:1048A000CF910895683818F0E8E7E60F25C0E62FA5
:1048B000F0E067FF12C0E058F10921E030E001C0EC
:1048C000220FEA95EAF72095DC0114963C911497A3
:1048D000322314963C93E0E00FC0E85DFD4FE49175
:1048E000EE2329F1E7FF08C0DC0114962C91149700
:1048F0002D7F14962C93EF7720E030E0EE2351F0DB
:10490000DC01A20FB31F16964C9116974E1302C0EE
:1049100016961C922F5F3F4F2630310579F7BC0168
:104920006C5F7F4F0E94DE2381E090E0089580E07D
:1049300090E00895FC011682178210861186128677
:1049400013861482BC016C5F7F4F0E94DE230895A2
:1049500087E195E00E94D3238BE095E00E94D62367
:104960000895A29FB001B39FC001A39F700D811D48
:104970001124911DB29F700D811D1124911D089568
:104980000E94B124A59F900DB49F900DA49F800D0F
:10499000911D11240895B7FF0C94C0240E94C024D7
:1049A000821B930B0895DB018F939F930E94C02479
:1049B000BF91AF91A29F800D911DA39F900DB29FBB
:1049C000900D1124089597FB072E16F4009407D03C
:1049D00077FD09D00E94752507FC05D03EF490951F
:1049E00081959F4F0895709561957F4F0895A1E23D
:1049F0001A2EAA1BBB1BFD010DC0AA1FBB1FEE1F59
:104A0000FF1FA217B307E407F50720F0A21BB30BA3
:104A1000E40BF50B661F771F881F991F1A9469F71F
:104A200060957095809590959B01AC01BD01CF017B
:104A30000895052E97FB1EF400940E94302557FD23
:104A400007D00E94F72407FC03D04EF40C943025C5
:104A500050954095309521953F4F4F4F5F4F0895AA
:104A600090958095709561957F4F8F4F9F4F0895DA
:104A70002F923F924F925F926F927F928F929F926E
:104A8000AF92BF92CF92DF92EF92FF920F931F935C
:104A9000CF93DF93CDB7DEB7CA1BDB0B0FB6F8940D
:104AA000DEBF0FBECDBF09942A88398848885F844D
:104AB0006E847D848C849B84AA84B984C884DF80BE
:104AC000EE80FD800C811B81AA81B981CE0FD11DA2
:104AD0000FB6F894DEBF0FBECDBFED010895EE0F07
:104AE000FF1F0590F491E02D0994AA1BBB1B51E117
:104AF00007C0AA1FBB1FA617B70710F0A61BB70B4E
:104B0000881F991F5A95A9F780959095BC01CD01F2
:104B100008958F929F92AF92BF92CF92DF92EF92C1
:104B2000FF92CF93DF93EC01688179818A819B8129
:104B3000611571058105910521F464E279ED8BE53C
:104B400097E02DE133EF41E050E00E941925490143
:104B50005A019B01AC01A7EAB1E40E94C0246B0199
:104B60007C01ACEEB4EFA50194010E94CE24C60EE8
:104B7000D71EE81EF91EF7FE06C081E0C81AD1084C
:104B8000E10880E8F80AC882D982EA82FB82C7017C
:104B9000B6019F77DF91CF91FF90EF90DF90CF909C
:104BA000BF90AF909F908F9008950E94892508959F
:104BB00086E091E00E948925089560930601709334
:104BC000070180930801909309010895F999FECF98
:104BD00092BD81BDF89A992780B50895262FF9993D
:104BE000FECF1FBA92BD81BD20BD0FB6F894FA9AD0
:0C4BF000F99A0FBE01960895F894FFCFCB
:104BFC0000001805200001000000FF000200020068
:104C0C000200020002000200020002000200020088
:104C1C0002000200020002000200028025000005D2
:104C2C00400AA1204EA50020244EA52C2330C012F2
:104C3C0000001A400AA1204EA5001B1E27522C234F
:104C4C00308025000005400AA1204EA50020244EEE
:104C5C00A52C2330004B000006400AD0009D4900D3
:104C6C007B289D492C233000E1000005400A4501BA
:104C7C00D7DC03B81E0EBF00232E48E801008A4083
:104C8C000A6001555502AD1E20000023C800E1004A
:104C9C000000000000010154582074696D656F75A7
:104CAC00742100456E746572696E67206164617071
:104CBC0074697665206368616E6E656C2073656CD3
:104CCC00656374696F6E2C207069636B696E673AEB
:104CDC00007363616E6E6572206D6F6465004F705A
:104CEC00656E4C52536E6720545820737461727405
:104CFC00696E672000206F6E20485720006D6F642E
:104D0C00756C65206C6F636B65643F0000070B0C62
:104D1C0010111500160A13223129000000000E1C78
:104D2C00AB1C9D1BC11BAA1B0A1CE41B0000000032
:104D3C00751EAB1C1B1E481E2D1E6A1E000000009B
:0A4D4C006B23AB1CE42352249A24CD
:00000001FF
